:02000000732863
:100008000800900022088400200839208413000585
:10001800181C2006031923281008031D1B2816087E
:10002800FF3E031C24280A30462016082428100AFC
:10003800FF3003192328100B2328170824289909AF
:10004800990C6E28A0003C200C080D0403196E289A
:1000580068208413200880066400322833288C0A1C
:1000680003198D0F302880066E28841780046E28A7
:10007800FF3A841780056E288001840AFF3E031D1D
:1000880040286E288F018E00FF308E07031C8F07D3
:10009800031C6E2803308D00DF30542048288D0162
:1000A800E83E8C008D09FC30031C5D288C07031882
:1000B8005A288C0764008D0F5A280C1863288C1C4A
:1000C80067280000672808008C098D098C0A031925
:1000D8008D0A080083130313831264000800831633
:1000E80004308500013086008B1783127E288B1B15
:1000F8000800A6297B200B167B2085017B20860122
:100108007B200C308400443040207B2006167B2066
:1001180001308F00F43047207B2086167B20013089
:100128008F00F43047207B2006177B2001308F009A
:10013800F43047207B2086177B2007308F00D03093
:1001480047207B2086017B2001308F00F430472038
:100158007B200530A2000430A000013098009601F1
:1001680097010130990024080520A4000318BE282F
:100178007B20A7287B2001308F00F43047207B208C
:10018800A60A7B20A4017B2064002608013C0319F1
:10019800F2287B2064002608023C031915297B20DD
:1001A80064002608033C031935297B2064002608CF
:1001B800043C031955297B2064002608053C0319D3
:1001C8007A297B2064002608063C031DF2287B2040
:1001D800A6017B20A4017B20A7287B207B20061377
:1001E8007B2086127B2006167B20323046207B201F
:1001F80004308C008D0106308400803026207B205E
:100208000530A2000430A000013098009601970143
:100218000130990024080520A4000318BE287B207B
:10022800FB287B2006137B2086167B2006127B206A
:100238000B308C008D0106308400803026207B2016
:100248000530A2000430A000013098009601970103
:100258000130990024080520A4000318BE287B203B
:100268001B297B2006177B2086127B2006127B2009
:1002780028308C008D0106308400803026207B20B9
:100288000530A2000430A0000130980096019701C3
:100298000130990024080520A4000318BE287B20FB
:1002A8003B297B2006177B2086167B2006167B20A1
:1002B80083160130860083127B20FF308C008D016D
:1002C80006308400803026207B200530A2000430D0
:1002D800A000013098009601970101309900240888
:1002E8000520A4000318BE287B2060297B208617E0
:1002F8007B2006177B2086167B2006167B20013084
:100308008F00F43047207B2086137B2006137B2048
:1003180086127B2006127B2001308F00F4304720A4
:100328007B200530A2000430A0000130980096011F
:1003380097010130990024080520A4000318BE285D
:100348007B207A29061386120612861301308F0045
:10035800F4304720A5016400153025020318C4298C
:1003680006178612061601308F00F4304720061350
:100378008616061201308F00F4304720A50FAF29EA
:0C03880086018B106400C6296300C829A0
:02400E00F53F7C
:00000001FF
